:10000000831600308100831200308B00831600308D
:100010008500F830860083128501860190013F300B
:100020009300B922140890009401930146203120D6
:100030003120252031204620252031202520462032
:1000400025202520252031205028061505308C003C
:100050000B308D00AE208D0B2A288C0B2828061122
:100060003C2806150F308C000B308D00AE208D0B18
:1000700036288C0B3428061105308C000A308D0090
:10008000AE208D0B40288C0B3E2808000A308C00D7
:100090000A308D00AE208D0B4A288C0B48280800B2
:1000A000861DBC28061E5728861E77285028061451
:1000B000861406158F0105308C000B308D00861ECE
:1000C000AB20AE208D0B61288C0B5D2806108610AE
:1000D000061105308C000A308D00861EAB20AE2044
:1000E0008D0B6D288C0B6B280F1877285028061F56
:1000F00099280614861406158F010F308C000B30DA
:100100008D00AE20061EA8208D0B81288C0B7F2829
:1001100006108610061105308C000A308D00061E70
:10012000A820AE208D0B8F288C0B8D288F18572878
:1001300050280614861406158F01AE20061EA8202E
:10014000061BA428861E9D280610861006118B28E3
:1001500002308F00080001308F00080032308E001E
:10016000B128B2288E0BB028080028308E00B8289D
:10017000B9288E0BB728080092228619BA298E2238
:1001800026221C22942283223F30910093010F30BB
:100190009500960108309200083097001F22CC2865
:1001A00014140310940D92031410F2200121970BE4
:1001B000DC2890228501C0281F22E9281410031092
:1001C000940D92031414F2201D21083097001F2271
:1001D000E9281010392108309700402139213921B0
:1001E0002520CC28920BF928C222D722910BFC287B
:1001F0004E2A0310940D0029930A083092009401AE
:10020000080006158F0105308C000B308D00861E0E
:10021000AB20AE208D0B09298C0B0529061105306A
:100220008C000A308D00861EAB20AE208D0B13296A
:100230008C0B11290F18DE28080006158F010F30CE
:100240008C000B308D00061EA820AE208D0B2529BA
:100250008C0B2129061105308C000A308D00061EFA
:10026000A820AE208D0B2F298C0B2D298F18D0287C
:10027000080014140310940D92031414F2200800C3
:1002800023308C000A308D00AE201F228D0B4429B4
:100290008C0B4229080094221C221018382A1410B2
:1002A0000310940D92031410920B57295D2903102B
:1002B000940D9203940D920B5729C22210089400BA
:1002C0003F309300C222850191016821702250289D
:1002D000922200309300B92208309200941F7129B5
:1002E000772992030310940D941F83297F29920389
:1002F0000310940D941F81297D29AF218429982111
:1003000084298B2184290800920B8829930A6B2960
:100310000310940D6E29061505308C000B308D00EE
:10032000AE202C228D0B90298C0B8E290611A4292E
:1003300006150F308C000B308D00AE202C228D0B5B
:100340009D298C0B9B29061105308C000A308D00ED
:10035000B5202C228D0BA8298C0BA62908000A3069
:100360008C000A308D00AE202C228D0BB3298C0B13
:10037000B129080094221018382AC221861B2F2A7E
:10038000A622BD29942200309300B92208309200A1
:10039000941FCB29D12992030310940D941FDD29BA
:1003A000D92992030310940D941FDB29D729112218
:1003B000DE29F621DE29E521DE290800920BE2295B
:1003C000930AC5290310940DC8290614861406152E
:1003D00005308C000B308D00AE202C228D0BEC29CB
:1003E0008C0BEA29061086100611062A06148614BC
:1003F00006150F308C000B308D00AE202C228D0B9B
:10040000FD298C0BFB2906108610061105308C0087
:100410000A308D00B5202C228D0B0A2A8C0B082A5D
:1004200008000A308C000A308D00AE202C228D0B83
:10043000152A8C0B132A0800861D1C2A0800861D0D
:100440004B29061ED028861EDE28080031202520D4
:1004500025202520312008008619080092228C01D1
:100460008D018E010610861006111C229422502840
:100470009422312025204620312031203120462071
:1004800046204620312025202520462025203120C9
:10049000462031204620252031205028922231202C
:1004A000252046203120312031204620462046207C
:1004B00025203120252046203120312031204620A2
:1004C0003120312046200530950096018501922289
:1004D0000F3085009222950B662A850183225028D1
:1004E0009222462031203120312046203120252003
:1004F000312046204620462025202520312031204D
:10050000252025200800403091009301FF30940001
:10051000C222930A910B862A101408002830952ACB
:100520000A30952A0530952A01308C0014308D0050
:1005300032308E009B2A9C2A9D2A9E2A9F2A8E0B4F
:100540009A2A8D0B982A8C0B962A080032308C0040
:100550002C221E308D0032308E00AE2AAF2AB02AF7
:10056000B12AB22A8E0BAD2A8D0BAB2A8C0BA82A8E
:1005700008008312130889008316081483120808E0
:100580009400080083168B13081583121308890042
:1005900014088800831655308900AA308900881411
:1005A0008B17081ED12A081208118312080016188A
:1005B000E22A950BE22A0310960C96151608850080
:0605C0000F309500080059
:02400E00F33F7E
:00000001FF
